:020000040000FA
:100000008A01D72C000000006400F000030EF1000C
:100010000A08F2000408F300831203138A110A127B
:100020009E2A8B138B1B11285E30AD0060305D283B
:100030008B138B1B18282630AD0027305D288B13BF
:100040008B1B1F281330AD0014305D288B138B1BC6
:1000500026288930AD000A305D288B138B1B2D2894
:10006000D130AD0004305D288B138B1B3428E83071
:10007000AD0002305D288B138B1B3B28F430AD00A4
:1000800001305D288B138B1B42284930AD000130B5
:100090005D288B138B1B49283130AD0001305D2862
:1000A0008B138B1B50282730AD0001305D288B133C
:1000B0008B1B57280530AD000130AE0023148B1781
:1000C00023185F2808008B138B1B6328BC30CF00DC
:1000D000BF30A8288B138B1B6A285E30CF0060309E
:1000E000A8288B138B1B71282630CF002730A82817
:1000F0008B138B1B78281330CF001430A8288B1358
:100100008B1B7F288930CF000A30A8288B138B1BCC
:100110008628A130CF000830A8288B138B1B8D2890
:10012000D130CF000430A8288B138B1B9428E830E3
:10013000CF000230A8288B138B1B9B283130CF00B7
:100140000130A8288B138B1BA2280530CF0001306B
:10015000D00023168B1708008E018F01C828DF30CE
:100160008E00BF30C72800308E00C030C728143042
:100170008E00FE30C728B8308E00FE30C728FA3017
:100180008E00FE30C728DF308E00FF30C7288F007A
:100190008B138B1BC828101463000C1CCC28101068
:1001A0000C108B17080000308A006C08820049345C
:1001B0004A34643465346634673474347534763460
:1001C00077346C346D34793459345A345B345C345C
:1001D0005D345E34EC34ED34EE34EF34FC34FD3415
:1001E000FE34FF34E4344B34C9345234C101D730C7
:1001F000EC00D3206002031DFF2803140800C10A8D
:100200001F30410203180629EC0AF9280310FE28C2
:1002100001308A002F0383120317E318033E831271
:10022000031382070534143423340A340F341E3484
:10023000FD030310FD0D7D0DA407031C2029A50A55
:1002400013308E2F0030A4000330A5000D308E2710
:100250006830A4003630A5000E308E2F8B138B1B18
:100260002E294B08031949294A08840083170008DE
:10027000B000840A0008B100A921031C4929CA0A58
:10028000CA0A60304A02031C47294030CA00CB0327
:10029000CB038B17080020304B02031962294A0850
:1002A0004B07840060300402031C5829E0308407A7
:1002B000831765088000840A66088000CB0ACB0A91
:1002C0000314632903100800831603130716871508
:1002D0007C2107127C2187118312031308008316E7
:1002E000031307127C2187157C2107167C218312BA
:1002F00003130800F8307D29FA30013E031D7D29E3
:10030000080083160313FA000830FD00FA0D0318E5
:100310008B2907128C2907167C2187157C218711D0
:100320007C21FD0B862907167C2187157C218312F1
:100330000313071AA1298316031387117C210310C5
:10034000A6298316031387117C2103148312031338
:1003500008006421B20132156E3081210318C929C9
:100360004C3081210318C929300881210318C9297B
:10037000310881210318C92930083107FF3A81214A
:100380000318C9296F213218F429B218F729031468
:1003900008006F210310C82981210318C9294C3096
:1003A00081210318C929300881210318C9296F2127
:1003B000C729831603130830FD0087157C2183129B
:1003C00003130314071AE5290310FA0D8316031308
:1003D00087117A21FD0BDD29071687157C218711EE
:1003E0007A2183120313080064214F30FD29642110
:1003F0005F30FD29B20164216F30812103180A2A80
:10040000831603138715831203131D2287190D2AE0
:100410005F1B062A6F2103101C2AD9216F21320885
:1004200003191B2A4E30321C5E30300731077A0226
:1004300003191B2A0B2A031408008B138B1B1D2A7C
:10044000831203170530EA000130EB008312031317
:100450005F178B170800A31E322A8830E500590861
:10046000E6004B290800A31E532A8030E5005A0EEF
:100470000F39E6004B21031C532A8130E5005A084E
:100480000F39E6004B21031C532A8230E500590E38
:100490000F39E6004B21031C532A8330E50059082D
:1004A0000F39E6004B2908006421A0308121031890
:1004B000542A080054223808FA003908FC00831333
:1004C000303084007A08812100088121840AFC0BE5
:1004D000642A6F29831603130830FD0087157C21D9
:1004E000831203130314071A762A0310FA0D8316D6
:1004F000031387117A21FD0B6E2A83120313080060
:100500008316031307127C2187157C2187117C2118
:1005100007167C295422380881216421A1308121C9
:100520008313303084003908FC006A227A08800086
:10053000840AFC0B9C2A6F298022952A8B1EAC2CE6
:100540000B1DAC2C0B11231CAA2AAD0BAA2AAE0B37
:10055000AA2A231044080319B72A023044020319B7
:10056000B52AC50BB72A0230C5002015B82A2011BC
:10057000A31DED2ACC0A3D304C02031DC52A0608F6
:10058000F0390319E92ACE00ED2A7A304C02031D16
:10059000CF2A0608F0394E02031DE92AED2AB730AA
:1005A0004C02031DD92A0608F0394E02031DE92A20
:1005B000ED2AF4304C02031DED2A0608F0394E02F4
:1005C000031DE92ACE1BE62AA318E92AA3144E0824
:1005D000CD0006080B108B15A311231EF42ACF0B98
:1005E000F42AD00BF42A23125F1FFF2A8312031769
:1005F000EA0BFF2AEB0BFF2A831203135F1383120C
:100600000313C01E0D2BD10B0D2BD20B0D2BC012C3
:10061000831603138C128312031383120317E60B42
:10062000F52BE70BF52BE830E6000230E7008312EC
:100630000313031086190314F90D7908031D222BE7
:10064000E313272BFF3C031D272BE3176313031032
:10065000051E0314F80D78080319332BFF3C031D06
:10066000342B5F15342B5F111F183C2BC0306707EC
:100670009F001F141F15F72B1F19F72BF401F5010D
:10068000670803195E2B0830670203194E2B1830D8
:1006900067020319562B1E08EE07ED2B1E08EE0706
:1006A000E311643E031C552BE315ED2B1E08EE07EA
:1006B0006315C83E031C5D2B6311ED2B1E08EE076E
:1006C00083160313C4004708F4070318F50A460805
:1006D000C700F4070318F50A4508C600F407031815
:1006E000F50A4408C500F4070318F50A0310F50CD1
:1006F000F40C0310F50CF40C83120313853058022C
:10070000031D882B0C08DA000D08D9003322BC2BFE
:1007100086305802031D9A2B831603130C0883128C
:100720000313DA00831603130D0883120313D90091
:100730003322BC2B87305802031DA32B0B08DA0091
:10074000D9013322BC2B88305802031DB52B2F084A
:10075000F400DA0110306219DA003E08AF00082117
:10076000D90033227408AF00BC2B84305802031D1B
:10077000BC2B7408D9002B22E3127408E401E31B9C
:10078000D42BD5145F3E0318C72BE316E02BF73E9E
:10079000031CE02BE40AF33E031CE02BE40AEF3ECB
:1007A000031CE02BE40AE02B493E031CE02BE40A87
:1007B000DF3E031CE02BE40AE73E031CE02BE40AC7
:1007C00062146416E31BE72B6412E412ED2BE412AF
:1007D000631DED2BE4160330E4040830E7072030F6
:1007E0006702031DF42BE7011F1083120313621E1F
:1007F000232CFF1B022CFF17831603130C30CE0093
:1008000083120313861C092C2319232C061F232C67
:100810000613E21B132CE217831203173130E20098
:1008200083120313232C83120317E20B212C831250
:100830000313FF13E2138A150A12EB268A110A1218
:10084000551583120313621B2E2C83120317E00B22
:100850002E2CE10B2E2C8312031362178312031725
:10086000631C372CE40B372CE50B372C63108312F9
:1008700003136318502CA21C542CE318462CE314C9
:1008800083120317D130E8000430E9008312031704
:10089000E80B522CE90B522C83120313A210542C98
:1008A000A214E31083120313231B63108316031394
:1008B000B70A08303702031C6A2CB70183120313EE
:1008C000A01D672CE319672C1030A006682C20129D
:1008D000831603133818752CB90B752CBA0B752CAD
:1008E0003814E830B9000230BA0083120313551DE2
:1008F000862CD51A862C9130F4001030F5008A151C
:100900000A169F278A110A12031855117F1E942C6C
:1009100083160313C80B922CC90B922C831203135A
:100920007F12F71283120313E21DAC2C7F1FA32C3E
:1009300083160313CA0BAA2CCB0BAA2C8312031306
:100940007F13E211AC2C7F17831603139630CA0075
:100950009930CB00831203138B188B108B1DB62C90
:100960000B1CB62C8B110B10A315CC018313831613
:1009700003138C1EC22C831203138C1EC22C8A11EB
:100980000A16F628831203130C1EC92C8A110A16A4
:10099000A7288A150A16572EB827BE277308840081
:1009A00072088A00710E8300F00E700E090020306C
:1009B0008300813081008E0100308C008D011B305E
:1009C0008500FF3086009B30870024309800563029
:1009D000990004309F00833092008312031340304B
:1009E0008B008C018D01103085005C3087000E304B
:1009F000900000309200910190309800C0309F002C
:100A00003B3094008A150A16812F83120317E830B1
:100A1000E6000230E70083160313FF30C400C50070
:100A2000C600C700B812C301831203135F1203305C
:100A3000E400E31263138330A000B8275030A10014
:100A4000BB276230A200BE2763148B138B1B252D9E
:100A5000C50A8B120B110C10831603130C14E8300B
:100A6000B9000230BA00FF30BC00BD00B814381520
:100A70008312031310148B110B1081010B118B16B1
:100A80008B1734202214BE2763127F18502D771A3B
:100A9000502DDF19502DF0278A110A12031C522DF8
:100AA00063167F101F201630B0007F30B100A327DF
:100AB000031C682DA827031C682DA921031C6B2D7E
:100AC0007A0ED800D81F6B2D8F30D805A3166B2D4A
:100AD0002210BE27412D6212DD01A030DE00C701C9
:100AE0001030C600C9013030C800CB014030CA0008
:100AF0008A150A1299208A110A127D0D8312031792
:100B0000E310031CE314831203138A150A166F2AD9
:100B1000A013A010262022218A150A125E278A110E
:100B20000A12631E872EAA30B0000130B9000430CB
:100B3000B8005A22A015A21762192017A310CD01E0
:100B4000DF19AC2D771AAC2D63120530FC00342070
:100B5000861FAE2DFC0BA72D6316B52DC827EA27DF
:100B60008A150A124E238A110A12C827EA278A1107
:100B70000A126408031DBE2D861DF62D02306F0279
:100B80000319DC2DD51FCB2D9B30E5000130E6008D
:100B9000DB278A110A128430E500E601DB278A117F
:100BA0000A128430E500E601DE278A110A12771A5C
:100BB000DC2D0130EF00FF119420E4278A110A1286
:100BC000861BDC2D231ADD2DDF118B138B1BE52DEE
:100BD00006080B108B15A310CD018B1702306F0286
:100BE0000319F52D8A150A16402BC8272E21E42754
:100BF0008A150A16E2258A110A12631F542EC401AF
:100C000023128130A000B8270130EF00981307139A
:100C1000E1278A110A124708031D082E8A150A12B5
:100C2000E5278A110A12E31AB52F621A342E621FC1
:100C3000342E6A209030E5008030E600DB278A11F0
:100C40000A12E1278A110A12861F2D2EF0278A1117
:100C50000A1203187C2E031C192E231A212E8A1522
:100C60000A12B3238A110A12F0278A110A120318F2
:100C70007C2EE31B442ED519132E8A150A12BE238F
:100C80008A110A12C827872EC82763138A150A12E9
:100C9000B5238A150A16E2258A110A12C827DF151C
:100CA000ED278A110A12052D5F196D2EE1278A1191
:100CB0000A128130E500E601DB278A110A12031CC3
:100CC000562EE1278A110A128530E500F030E60041
:100CD000DB278A110A12031C612EED278A110A12E2
:100CE000A31C4A2FCD1FBE2E9B20861F7A2E231AAF
:100CF000752E7C2ECD13BE2EA3105F169420861B5E
:100D00007E2E231A7F2E9530E500E601DB278A111F
:100D10000A16B3248A110A125F120C306F020319EB
:100D2000A52EFF1D052D9330E5006F08E600DB279B
:100D30008A110A12DE278A110A12A0108D20E427D8
:100D40008A110A12231A9F2EB72E831603133B080B
:100D500083120313023C031DB02E77160230B12E0E
:100D60000130EF006408031D052DE31B052DA310C2
:100D70009420861BB82E231AB92EF62D4D1F2C2F2A
:100D80001430FC003420061BDF2E77139630E5006C
:100D9000E601DB278A110A120130B900B0010230E6
:100DA000B8005A228A150A12AF238A110A12C827DC
:100DB000EA278A110A123420CD1B7C2E482FFC0B07
:100DC000C22E8A150A12DD238A110A12C827EA27C1
:100DD0008A150A12172717278A110A123B20A430F6
:100DE000BB004C30BA008A150A123327B030BA0063
:100DF0002B278A110A12061B002F4220061F052FDF
:100E00008618FB2E49208618FB2E8B138B1B052F73
:100E1000EA278A150A1600208A150A12DF238A118A
:100E20000A12C827EA278A150A1600208A110A1210
:100E3000E4278A110A1277179630E5000130E600A0
:100E4000DB278A110A12031C182F0130B000B900E9
:100E50000230B8005A22D22E4D1E432F1430FC000F
:100E60003420061A362F861E482F2E2F861E2E2F30
:100E7000FC0B302F013083160313BB0083120313C6
:100E80000730EF00572FCD1E482F0630EF00482FB8
:100E9000A310CD01401E572F4012F620031CF62D43
:100EA00001306F02031D572F8A150A1687280A3052
:100EB0006F020318052D6F080319052DAF008A1561
:100EC0000A162D2EA31B7F2F06306F020319812FC8
:100ED00001306F02031D7E2F9330E5006F08E6009E
:100EE000E4278A110A12DB278A110A12031C702FC9
:100EF000DE278A150A16B8278A110A12F62DA313BF
:100F00007C2E631B7E2F831603133B08831203136F
:100F1000093C03197E2F0C30EF007C2EFD00A60C3F
:100F2000A50CA40CA215031CA211BE272215BE27D6
:100F3000FD0BA02F2216BE272211BE272212BE2F84
:100F40002211BE278F2F6421B20132144E30AD29F9
:100F50006421B201B2145E30AD29B20164214F3078
:100F6000FD29B20164215F30FD298A150A163F2F41
:100F70008A150A1652288A150A165C288A150A1636
:100F8000662808008A150A16C0248A110A127E2FC4
:100F9000E4278A110A12621AC82F83120317C83075
:100FA000E0000130E10083120313E4278A110A12E2
:100FB000621FD52F08008A150A12FD2B8A150A1206
:100FC0001C2C8A150A12612C8A150A12602C8A15AB
:100FD0000A12842C8A150A12F82E8A150A16A52ED2
:100FE0008A150A12AB2F000000000000000000006C
:100FF00000000000000000000000000000000000F1
:101000008A150A1600288A110A12332A8A110A122E
:10101000B12F8A110A1264298A110A12F6288A1538
:101020000A16C02C8A150A16A52E8A110A122E2914
:101030008A150A1687288A110A126A288A110A1242
:1010400071288A110A1278288A110A127F288A11B7
:101050000A125A2A2030B00009205E308A110A1282
:10106000CC218A150A12031C4B2806208A150A1265
:10107000031C4B287A08D700D90089305802031D79
:101080004928DA018B138B1B422803208B178A1502
:101090000A120314080003104A282130B000092066
:1010A0005E308A110A12CC218A150A12031C4B28C1
:1010B00006208A150A12031C4B287A08FD003C28DA
:1010C00023304E2824304E2827304E2828304E28F2
:1010D00026304E282130B00009204E308A110A12E5
:1010E000CC218A150A12031C8D288A110A12AD27F9
:1010F0008A150A12031C8D287A08FD00D9008A304F
:101100005802031D8B28DA018B138B1B84280320C4
:101110008B178A150A120314080003108C2822303A
:101120006B2823306B2824306B2827306B2828301D
:101130006B2829306B2825306B282A306B282B3000
:101140006B282C306B282D306B282E306B282F30DD
:101150006B285618E728D60156140230E600E4281A
:10116000D618E728D601D6141230E600E42856191E
:10117000E728D60156152230E600E428D619E728DC
:10118000D601D6153230E600E428561AE728D601F3
:1011900056164230E600E428D61AE728D601D616BD
:1011A0005230E600E428561BE728D6015617623075
:1011B000E600E428D61BE728D601D6177230E600F1
:1011C000E428D601F030E6008530E500FD23080074
:1011D000831603133817B813F62883160313B817AA
:1011E0003813F628831603133813B8138312031326
:1011F000401E002940120C208A150A1203181828D4
:10120000602415202E212E212E218A150A120F204E
:101210008A150A16E2258A150A12031C30291220A3
:101220008A150A1203306F02031D3029A31C1A29E4
:10123000CD1B2F2983160313381F24298312031370
:10124000FD23031CF8282B29B81F2B298312031315
:101250001C24031CF8288312031303140800A3178B
:1012600003102E296217423095000C30970012159A
:101270009330E5000330E600E820031C472AED2008
:10128000031C472AF220031C472A9B20031C4229E7
:101290007D08031D42298A150A16B8278A150A12E5
:1012A000F220031C472A2A2057187229571A72293C
:1012B000D719722995207D0803196F29621E6129AB
:1012C000F82600208A150A128423D6011D23F22055
:1012D000031C472A231A67297D1B362A252AA920A1
:1012E00090235029621E7529F82600208A150A12BB
:1012F0009522031C152AE1208730E500E601ED2048
:10130000031C472A8030E5008030E600E820031CFB
:10131000472A1E208A150A12F220031C472A231A84
:101320008C298030E500E601E820031C472AC02311
:10133000F220031C472A621A98298A150A160020EF
:101340008A150A1283160313CC018312031321207A
:101350008A150A126024231AAA298830E500E601BA
:101360001C241B208A150A12F220031C472A622023
:101370007D0D031CF0297D080739FB0005307B0239
:101380000318C9298230E5007B08E600E820031C29
:10139000472A21208A150A12F220031C472A231A01
:1013A000CC29C023F220031C472A621AD2298A15AD
:1013B0000A1600208A150A12F220031C472AA720C9
:1013C000031CDC297D084039031DDC298316031327
:1013D000CC0A4C0883120313053C0319F229A729F0
:1013E000231AB4298430E500E601ED20031C472AC6
:1013F0008230E5001030E600E820031C472AC520B3
:10140000B12360244908031D012AF220031C472A46
:101410004D2010307D02031D052A8730E500013084
:10142000E600ED20031C472A162AC520F220031CE3
:10143000472A621F162A8A23A222F220031C472A67
:10144000231A1D2AD601D71D362AD3208A23D22259
:10145000F220031C472A231A282AD6012A205718CB
:10146000152A571A152AD71D6F29252AB7208A232E
:10147000D222F220031C472A231A392AD6012A2015
:101480005718152AD719152A571E6F29362AE12011
:1014900061248130E500E6011C248730E500E60187
:1014A0001C246024842415202E212E212E218A150F
:1014B0000A12621E682A8B138B1B5B2AF826831282
:1014C0000317D130E0000430E100831203138B17BF
:1014D00012119701A31B922A07306F020319922A57
:1014E00009306F020319922AE31B782A631B922AA0
:1014F0008430E5000C30E60001306F020319812AC8
:10150000E6016024FD23031C812AA31B922A602488
:10151000A720031C882A7D08F039031D872A8A1119
:101520000A121F208A110A12622F84244908031DFF
:10153000952A8A110A16E0228A150A12031C952A96
:101540007D0D08000830F123AF00A62A0A308A007A
:101550008B138B1BA82A0310AF0D2F0D8207E830C9
:10156000CF000130CE2AD130CF000330CE2AA130B7
:10157000CF000730CE2A7230CF000B30CE2A423057
:10158000CF000F30CE2A1330CF001330CE2AE330F5
:10159000CF001630CE2AB430CF001A30D000231638
:1015A0008B1708001030F123AF00002B0000000063
:1015B000000000000000000000000000000000002B
:1015C000000000000000000000000000000000001B
:1015D000000000000000000000000000000000000B
:1015E00000000000000000000000000000000000FB
:1015F00000000000000000000000000000000000EB
:101600000B308A008B138B1B022B0310AF0D2F0D99
:101610008207D130CF000330CE2AA130CF0007306F
:10162000CE2A7230CF000B30CE2A4230CF000F309E
:10163000CE2A1330CF001330CE2AE330CF0016303D
:10164000CE2AB430CF001A30CE2A8530CF001E30DB
:10165000CE2A5530CF002230CE2A2630CF00263079
:10166000CE2AF630CF002930CE2A9730CF00313045
:10167000CE2A3830CF003930CE2ADA30CF00403091
:10168000CE2A4B30CF004C30CE2ABD30CF00573061
:10169000CE2A2315E216512B2311502B003023158F
:1016A000E212621A512B621F512BE6008A30E500CC
:1016B00060241C24031C582B602447084907031D81
:1016C0005C2B68207D1C612B6420831603137D082E
:1016D000B500831203136620831603137D08B6003A
:1016E000831203130727831603133508831203138A
:1016F000BA0083160313360883120313BB00222794
:101700000314832B03100800621A842B621F842B9E
:1017100001304F2B621A822B621F822B21304F2BFC
:10172000621A822B621F822B02304F2B621A822B8D
:10173000621F822B03304F2B771F822B04304F2BDD
:1017400077139630E500E601FD230130B900B001C2
:101750000230B80027208A150A1205304F2B0530B9
:101760004C2B06304F2B0730492BD510A0108A1177
:101770000A123B208A150A1208304F2B09304F2BD2
:101780000A304F2B0E304F2BDF1A0800DF1683165E
:101790000313AA30CD00831203130F304F2B1030E8
:1017A0004F2B11304F2B12304F2B13304F2B143047
:1017B0004F2B15304F2B16304F2B1730492B18302D
:1017C000492B19304F2B1A304F2B1B304F2B1C300D
:1017D0004F2B1D304F2B1E304F2B1F304F2B2030E7
:1017E0004F2BFD006E080107FC007D080319FC2B40
:1017F000FC020318F82B7C0708008B138B1BFD2BB6
:10180000D516203047020319182C460847078400D4
:1018100030300402031C0E2CE03084078317650867
:101820008000840A66088000C70AC70A0314192CBE
:101830000310D5128B1708008B138B1B1C2C55170C
:10184000103049020319372C4808490784004030FA
:101850000402031C2D2CF0308407831765088000D8
:10186000840A66088000C90AC90A0314382C0310C8
:1018700055138B17080002305D0203195C2C03100E
:101880005D0D5D075E07031C462CFA3E8400A63002
:101890000402031C4D2CFA30840783136C0880006B
:1018A000840A6D08800084030007A438840A840A2F
:1018B0008000DD0A03140800A31B5A2C03105B2CC4
:1018C00055148B138B1B612C47080319802C460879
:1018D000840083170008B000840A0008B1008A1150
:1018E0000A12A3278A150A12031C802CC60AC60AEC
:1018F00030304602031C7E2C1030C600C703C703DD
:101900005518842C8B17080055108B138B1B852CB6
:1019100049080319A42C4808840083170008B00064
:10192000840A0008B1008A110A12A8278A150A122F
:10193000031CA42CC80AC80A40304802031CA22C6D
:101940003030C800C903C9038B17080060240F207A
:101950008A150A16E2258A150A12031CBF2C0630C6
:101960006F02031DBF2C64080319BF2CA31CBC2CE1
:10197000CD1BBE2CCD1AC12C03140800A3170310D5
:10198000BD2C0130EF00BF2C60240F208A150A16F1
:10199000E2258A150A12031CD92C06306F02031D9A
:1019A000D92CA31CD52CCD1BD92C621AC42C031402
:1019B00008000310D82CD513B0010130B900033052
:1019C000B80027208A150A12C401A017A011A2137B
:1019D0002013E523C424031CB82E621EF02CF82625
:1019E00000208A150A12E723C424031CB82E8A118A
:1019F0000A1294208A150A12861AF72C231AFC2C34
:101A0000A310CD019330E5000630E6006024FD23ED
:101A1000031C062D60241C24031C0A2DE9276024C6
:101A20006A20D51DE82E031C0F2D06307D02031DF4
:101A30000F2D8230E5006230E6006024FD23031C98
:101A40001D2DE923C424031CB82E621E282DF82660
:101A500000208A150A12EB23C424031CB82EA624E6
:101A6000031CB82EA720031C322D7D083039031D1E
:101A70002F2D8130E5000330E6006024FD23031C98
:101A80003D2DED230430FC008530E5002330E600D9
:101A9000FD2321208A150A12A624031CB82E231A1E
:101AA0004C2D8530E5006330E600FD2321208A15AA
:101AB0000A12A624031CB82E231A592DFC0B442D00
:101AC0008530E500F130E600FD23C424031CB82E68
:101AD0008230E5004030E6006024FD23031C6C2DBD
:101AE0008230E5005030E6006024FD23031C742D95
:101AF0008230E5001330E6006024FD23031C7C2DBA
:101B0000A624031CB82E47084907031D802DA624D0
:101B1000031CB82E621A8E2DC424E123A720031CB7
:101B20008E2D7D088039031D872D621A8E2D813000
:101B3000E5000330E600FD2321208A150A12A624C1
:101B4000031CB82E231A9F2D1E208A150A12A624C4
:101B5000031CB82E231AA72D21208A150A12A624A9
:101B6000031CB82E231AAF2D8230E5004030E6006A
:101B70006024FD23031CB82D8230E5005030E600C0
:101B80006024FD23031CC02D8030E5008030E6007A
:101B90006024FD23031CC82D21208A150A12A624C7
:101BA000031CB82E231ACF2D8230E5001630E60034
:101BB0006024FD23031CD82DA624031CB82E621A12
:101BC000E32DC424E323A624031CB82EA720031C62
:101BD000E32D7D088039031DDC2D621AE32D803052
:101BE000E5003030E6006024FD23031CF32D2120A6
:101BF0008A150A12A624031CB82E231AFA2D823045
:101C0000E5006630E6006024FD23031C032EA624B5
:101C1000031CB82EA720031C072E7D083039031D96
:101C2000072E8A110A1218208A150A120530FE00A2
:101C30008530E5002230E6006024FD23031C182EC9
:101C40008030E5002130E6006024FD23031C202EB7
:101C5000602447084907031D282ED52324208A1510
:101C60000A12A624031CB82E231A312EA624031C04
:101C7000B82E9320031C392E02307D02031D362E10
:101C80008030E500E6016024FD23031C432E8A1109
:101C90000A127F208A150A12A624031CB82E231AC2
:101CA0004C2E621E542EF82600208A150A1285300A
:101CB000E5006230E6006024FD23031C572E8030CF
:101CC000E5001230E6006024FD23031C5F2E602433
:101CD00047084907031D672ED72324208A150A12B7
:101CE000A624031CB82E231A702EA624031CB82E7B
:101CF0009120031C782E02307D02031D752E80304A
:101D0000E500E6016024FD23031C822E8A110A12DD
:101D10007F208A150A12A624031CB82E231A8B2EA4
:101D2000621E932EF82600208A150A12FE0B182E2A
:101D30008530E500F130E600FD238230E5003630E5
:101D4000E600FD23602447084907031DA22EA624B0
:101D5000031CB82E9320031CAA2E02307D02031D03
:101D6000A72E1E208A150A126024231AB42E192DBC
:101D7000C40161244708031DB92E9530E500E60132
:101D8000FD2361244708031DC12E621ED42E8B1330
:101D90008B1BC72EF82683120317D130E0000430C6
:101DA000E100831203138B178A110A1294208A15FB
:101DB0000A12861AD42E231AD92EA310CD0101306F
:101DC0006F02031DE52E7716E82E8A110A12622F84
:101DD0008A110A12052D6213831203172630E000C0
:101DE0002730E100831203136212231FA0120800A0
:101DF000EB26231B032F61249130E5001030E60011
:101E0000FD23031CFB2E1030BA002B270800E21A1A
:101E1000162F60249130E5001130E600FD23031CED
:101E2000092F602447084907031D112FA0162030F1
:101E3000BB000030BA0033278A110A122D208A1500
:101E40000A12080062165511E030BB073327F03044
:101E5000BA002B27080021138A110A12BB278A1502
:101E60000A1246273F2F21138A110A12BB278A150F
:101E70000A1246273B08BA003D08BC004627211736
:101E80008A110A12BB278A150A1208000830EB00D3
:101E9000A116BA0C031CA1128A110A12BB27A117A2
:101EA000BB270314061D0310BD0CA1138A110A12CF
:101EB000BB278A150A12EB0B482F08008030A400BC
:101EC0002430A5000530A6003E08AF008A110A1292
:101ED0000821FD008A110A1218218A110A123420E1
:101EE0002030A4001A30A5000330A6003E08AF0041
:101EF0008A110A120821FD008A110A1218218A1576
:101F00000A1208000F308A00430382070F34083496
:101F1000053402340034C300F030A1058227A10447
:101F20008A110A12BB278A150A12080009205E309E
:101F30008A110A12CC218A150A120800FB30FD0012
:101F4000FC01061EA92FFC0FA12FFD0FA02F5F146F
:101F5000AB2F5F10DF10F630FD00FC01861FB62F9F
:101F6000FC0FAE2FFD0FAD2F031408000310B52F8B
:101F700060248830E500E6011C24031CB82F60248F
:101F800015208A150A12470849074B07031DBF2F62
:101F90008A150A1262208A150A128B305802031D14
:101FA000BF2F7D08D900DA018B138B1BD42F0320A0
:101FB0008B178A150A12BF2F0F308A002F0882074D
:101FC00006340834023407340334FF30EA2F0F306C
:101FD000EA2F0A308B138B1BEA2F83160313C000E2
:101FE00083120313D5158B170800000000000000B2
:101FF00000000000000000000000000000000000E1
:102000000130F6000830F500F40C0318013EF50B22
:102010000428F60B14280F3C031810280314112869
:1020200003100800F60102280C3C031C1028013C98
:10203000031C10280E288B138B1B1B28ED0CFD0C8A
:10204000ED0CFD0C0314FD0C0314FD0CED0CFD0C4C
:10205000ED0CFD0C0314FD0CED0CFD0CFC01ED0C66
:10206000FC0CED0CFC0C0310FC0C0310FC0CED0C38
:10207000FC0CFC0CFC0C7C0CEC047D08ED008B17BC
:1020800008008B138B1B4128E00DE00DE00DE00DE7
:10209000FD0DE00DE00DE00DFD0DE00DFD0DE10D80
:1020A000FD0DE10DE10DFD0DE10DFD0DE10DE10D6C
:1020B000E10DFD0DE10D7D0DE1008B1708008A1586
:1020C0000A12FD2B8A150A121C2C8A150A123B2CA7
:1020D0008A150A12602C8A110A1278288A150A16A3
:1020E00066288A150A126A288A150A12A7288A15EC
:1020F0000A124D288A110A127F288A110A12332ADD
:102100008A150A16C02C8A150A16232E8A150A1259
:10211000A02B8A150A12F82E8A110A1294288A1501
:102120000A16A52E8A150A16282F8A110A12F628D1
:102130008A110A125A2A8A150A129E278A110A1629
:1021400008008A150A163F2F8A150A16872877185D
:10215000B228F718BD287719C9285D080319F32894
:102160007714DB01FF309900DB0A05305B02031DA9
:10217000F3287710F714DB01F3284C309900DB0AC1
:1021800003305B02031DF328F7107715DB01DC0138
:10219000F3285E085C078400831300089900DC0ABA
:1021A00003305C02031DF328DC01DB0A03305B0211
:1021B000031DF32880305802031DE9285E088400BF
:1021C00083130008DA00840A0008D9007D208A11F0
:1021D0000A167711DD030330DE07A6305E02031D09
:1021E000F328A030DE008A110A12C92C981CFC28A2
:1021F000181200001816832A401C36293F08840054
:1022000083131A088000F4000020031C832AC01ADC
:102210000E29C0166230D1000130D200BF0AC20AB6
:10222000083042020318832A2A303F02031C8B2AFB
:102230002708A4002808A5002908A6002408A50648
:102240002509A40525082605A404FF302402031946
:102250002F292808A7002908A800BF038B2A4010AF
:102260004015C0142430BF00C2018B2AC01C642951
:10227000C20A073042020318832A3F0884008313EE
:102280001A088000F400401D4829002003188B2AFA
:102290000008F4001220031C95294011BF0A2730C2
:1022A0003F02031C8B2AC0102408A5062509A4059B
:1022B00025082605A4044C302402031D952924304A
:1022C000BF00C01563148B2AC01D892A3F088400F3
:1022D00083131A088000BF0A2D303F02031C8B2A8B
:1022E000C0012408DA00A7062709A40527082A0543
:1022F000A4042508D900A8062809A50528082B0547
:10230000A5042608A9062909A60529082C05A6045E
:1023100083305802031D8F297D208A110A16240854
:102320002507A43826020319A429EA0A0319E90A91
:1023300082305802031D832A6A08D9006908DA002E
:102340007D208A110A16832A40162408E000DA004C
:102350002508E100D90081305802031DB2297D20F3
:102360008A110A165D306002031DC0296108013917
:102370000319BD29201762157A2A201362117A2ABF
:102380005A306002031DD729F71A792AF7168316E7
:1023900003133830C8003A30C900831203137F1684
:1023A000C40A03304402031D792AC401792A5F302C
:1023B0006002031DE029E118F7126118E211792A81
:1023C00053306002031DE6295F12F029523060028B
:1023D000031D332A55168A150A16BF268A110A16B6
:1023E000401283160313D10A03305102031CF9294A
:1023F000D101510883120313FF3E03191A2AFF3E2D
:102400000319142A4C30ED00F71AED14D51BED1604
:1024100062196D16E21D122A6D1404306F02031D3D
:10242000122AED17CA302E2A640803394C38ED0001
:10243000CC302E2A09306F02031D242A8316031381
:102440003B0883120313252A6F08ED006D0EED047F
:102450003C30ED04621D6D12ED11CB30EC006520B7
:102460008A110A16832A49306002031D622AA310CA
:1024700049306102031D3E2A01305D2A4B30610262
:10248000031D452AA72703305D2A4A306102031D38
:102490004B2A02305D2A4D306102031D512A05305E
:1024A0005D2A4C306102031D582AAD2704305D2A95
:1024B0005F306102031D5F2A0730EF00612A40127E
:1024C000832A792AE4306002031D782A4A306102A7
:1024D000031D6C2A7F15772A49306102031D722A79
:1024E000FF14772A4B306102031D772AFF167A2AE0
:1024F0007A2A4012C930EC0060086107A438ED0068
:1025000065208A110A164014C012C2012730BF008C
:102510008B2A1A08832A8A110A12C22C83160313E3
:102520004F149A2A83160313CF144F109B2A831635
:1025300003134F10CF1083120313401EA52A40121D
:1025400095208A110A160318A42880208A110A16D9
:10255000831603134F18B72ACF18B72A8312031311
:102560008A150A16E2258A110A16031CDE2A83122E
:1025700003138F208A110A1605306F02031DDE2A0D
:10258000A31CC42ACD1BDD2A831603134F1CD02A9B
:10259000831203135F208A110A16031C9D2AD92A6D
:1025A000CF1CD92A8312031362208A110A16031C36
:1025B0009D2A8312031303140800A3170310DC2AB7
:1025C0002230B000B1008A150A1296278A110A1625
:1025D000031C0B2B8A110A12B1278A110A16031C3D
:1025E0000B2B7A08FD00D90089305802031D002BFF
:1025F000DA018B138B1BF92A7D208B178A110A169F
:102600007D0D031C092B8030E500E60162208A1154
:102610000A160314080003100A2B9330E500053056
:10262000E6009222031C0D2C8E22031C0D2C9722F7
:10263000031C0D2C74208A110A16031C172B7D080D
:10264000C039031D172B9722031C0D2C77208A11EC
:102650000A1610307D02031D232B8730E500013060
:10266000E6009222031C0D2C4D1F3C2B4D13A31092
:1026700086208A110A16712B9722031C0D2CE0224A
:10268000031C342B7D0D031C342BB1278230E50055
:102690007E08E6008E22031C0D2C8730E500E60143
:1026A0009222031C0D2C8230E5001530E6008E22AC
:1026B000031C0D2C9722031C0D2C47084907031DF2
:1026C0005A2B74208A110A16031C5A2B7D08C03914
:1026D000031D5A2B8A150A12962303189C238A116C
:1026E0000A166B208A110A169722031C0D2C621AF7
:1026F000712B231A742B8930E500E6019222031C0A
:102700000D2C8830E500E6019222031C0D2C831667
:102710000313CC01831203138A110A126A208A114F
:102720000A164D1F992B4D13A31086208A110A16E5
:10273000BF2B9722031C0D2C8A150A1262208A11C6
:102740000A167D0D031C0A2C7D080739FB00053095
:102750007B020318B22B8230E5007B08E6008E2254
:10276000031C0D2C6B208A110A169722031C0D2CBA
:10277000231AB52B8A150A12C0238A110A1697222A
:10278000031C0D2C47084907031DBF2B621ABF2BE2
:102790008A150A1600208A110A169722031C0D2C8E
:1027A00074208A110A16031CCD2B7D084039031DA5
:1027B000CD2B6B208A110A169722031C0D2C231A8D
:1027C000DC2B8830E500E6019222031C0D2C8316D9
:1027D0000313CC0A4C0883120313053C031D8C2BF6
:1027E0008430E500E6019222031C0D2C8230E500C6
:1027F0001030E6008E22031C0D2C9722031C0D2C9A
:1028000074208A110A16031CFD2B7D088039031CD5
:10281000FD2B232B231A912BF02B8730E500E601AB
:10282000D127DA27E327621E242C8B138B1B152C50
:1028300089208A110A1683120317D130E000043070
:10284000E100831203138B17A31B292C8A110A1290
:1028500018208A110A12622FD513C401D51B352CFA
:102860008330E500E601C827EC279330E500073008
:10287000E600C827D12780208A110A168316031381
:102880000314B81C0310381D0310831203138A119C
:102890000A12031CF62D8A150A129B208A110A16A9
:1028A000031C3B2C7D08031D3B2C831603130730B0
:1028B0003B020319652C831203138A150A1609308B
:1028C0006F020319CE2D8A110A16831203130B30DF
:1028D000EF008230E5001330E600C82768208A1137
:1028E0000A1674208A110A16031C6E2C7D08803982
:1028F000031D6E2C8230E5004030E600C827823090
:10290000E5005030E600C8278430E5007730E60067
:10291000C82768208A110A1674208A110A16031C17
:10292000892C7D087C39031D892C7830B00001305A
:10293000B9007030B80098208A150A121727172797
:102940008A110A123B20A430BB004C30BA008A1511
:102950000A1233278A150A12F8268A110A1226202B
:102960008A110A16A1286F0883160313BB0083126D
:1029700003137712C40102306F020319C22CE31F44
:10298000A128C42C0A30C72CF127A0170C30EF0067
:10299000A01489208A110A122D208A110A162312E6
:1029A0009330E5006F08E600C827D12722136E2078
:1029B0008A110A16E3278B17631B2E2DA01B2E2DC1
:1029C0005F1D2E2DE31AA1288F208A110A16621C82
:1029D000F82C62109030E5006408E600551AF22CDD
:1029E0004030F42CEF278030E6045F208A110A166D
:1029F000A01B172D5F1D172D401E042D4012952082
:102A00008A110A160318A4285F1C172DDF18172D2A
:102A1000DF149730E50083160313D003500D023006
:102A20000318D000500883120313E6005F208A15B4
:102A30000A1261248A110A169B200318A12D0A305C
:102A40006F020319DC2C0C306F0203192E2D8A152E
:102A50000A1696268A110A167716B32D5F1255129A
:102A6000A014AD27E31B982D9430E5000130E6005B
:102A7000C827A2126E208A110A16DA27F127A0179A
:102A80008A110A12B8278A110A168B138B1B452D3F
:102A9000E31AA1288B138B1B4A2D98130713831657
:102AA00003138C128312031386195B2D06080B1077
:102AB0008B1563000B109B200318A12D0C18642D9F
:102AC0008B1700000000482D0B15831203170130EF
:102AD000E6000130E700831203138B1783208A116D
:102AE0000A16E31B982D631B3E2D0C306F02031951
:102AF000A128A0137A208A110A169B200318A12D61
:102B0000231A7D2D8A110A1222218A150A125E27A4
:102B100098178A110A127120E21963208A110A1685
:102B20008F208A110A169B200318A12D5F1D9C2D52
:102B300092208A110A16E22CE31B982D231A902D5D
:102B40003E2DA01BB32D5F1DB32D551EB32DF127B8
:102B5000A0170C30EF008C208A110A16861BAB2DB3
:102B6000231AAE2D982D8A150A162D278A110A16BA
:102B70008F208A110A167F14080080208A150A16F1
:102B8000E2258A110A16031CD32D8F208A110A16FA
:102B900004306F02031DD32DA31CD02DCD1BD22DCD
:102BA00003140800A3170310D12DDF12E214933091
:102BB000E5000430E600BD25031C612F62208A1168
:102BC0000A16031CDB2DBD25031C612F5F208A1113
:102BD0000A16031CE32DBD25031C612F4708490776
:102BE000031DEB2DBD25031C612F74208A110A16CD
:102BF0007D084039031DF22DBD25031C612F772070
:102C00008A110A1610307D02031DFC2DC401AD2768
:102C10008A110A1226208A110A16A21E372EBD25F5
:102C2000031C612F9830E500E6015F208A110A1627
:102C3000031C0F2EE21C272E8A150A12E7278A1181
:102C40000A16BD25031C612FD519212EE210BD25C2
:102C5000031C612F9430E500E6015F208A110A16FB
:102C6000031C272EA2126E208A110A16DA278B1750
:102C70008830E500E60162208A110A16E327DF1397
:102C80008B138B1B402E98130713831603138C1280
:102C90008312031306080B108B158B100B166300A1
:102CA0008B185A2E0B185A2E0C185C2E8B170000FE
:102CB0000000402EDF176B2E0B1583120317013017
:102CC000E6000130E700831203138B1783208A117B
:102CD0000A16631B612FA01F7F2EA0137A208A1172
:102CE0000A16061CDF17BD25031C612F231A712E3F
:102CF0008A110A1222218A150A125E2798178A1150
:102D00000A1271208A110A16061CDF178F208A11F9
:102D10000A16BD25031C612F5F1D9F2E551E912E87
:102D2000A727061CDF17DF1BA62EBD25031C612F5E
:102D3000A01B062E5F198E2E5512A017062E5512B7
:102D4000DF1BA62E231A842EA017062E8B100B1223
:102D5000A7278A110A126A208A150A1262208A118C
:102D60000A167D0D0318B72E231AAC2EE02E7D080F
:102D70000739FB0005307B020318E02E92208A11F0
:102D80000A16BD25031C612F8230E5007B08E60092
:102D90005F208A110A16031CC12EBD25031C612F5A
:102DA00047084907031DCD2EBD25031C612F742044
:102DB0008A110A16031CD42E7D084039031DD42E17
:102DC000BD25031C612F8730E5000130E60062203D
:102DD0008A110A16031CE02EBD25031C612F8930C1
:102DE000E500E60162208A110A16031CEC2E8C20F5
:102DF0008A110A1668208A110A1647084907031D16
:102E0000F72E231AFA2E8A110A1263208A110A1643
:102E1000BD25031C612FE022031C032F7D0D031829
:102E20002C2F2C307D020318182F231A082FE02E88
:102E3000BD25031C612FE022031C182F7D0D0318F4
:102E40002C2F11307D020318182F8A110A121F200F
:102E50008A110A16DF13742F7D08B12792208A1178
:102E60000A16BD25031C612F9830E5000130E600ED
:102E70005F208A110A16031C312F0230C400E215AC
:102E80008230E5007E08E6005F208A110A16BD2523
:102E9000031C612F47084907031D472FBD25031C4D
:102EA000612F74208A110A16031C402F7D084039B7
:102EB000031D4E2F8A150A12C223C4238A110A1633
:102EC000742F2312C401AD2792208A110A1668209C
:102ED0008A110A169830E5000130E6005F208A1159
:102EE0000A16031C672F0D2CBD25031C612F621AC7
:102EF000742FC4019830E500E6015F208A110A169C
:102F0000A21E932FBD25031C612F9430E500E6011E
:102F10005F208A110A16031C822FA2126E208A11CA
:102F20000A168B17DA276B208A110A1677208A1166
:102F30000A1610307D02031D932F231A962F883016
:102F4000E500E60162208A110A16DF138E2EA0101A
:102F5000A015A217621920170800A011A2132013B0
:102F600008000130FE009D307D02031CC72FFE0AC1
:102F7000BB307D020318C72FFE0AA7307D02031C59
:102F8000C72FFE0AB1307D020318C72FFE010800CB
:102F900068208A110A165F208A110A16031CC82F9E
:102FA000080068208A110A1662208A110A16031C7A
:102FB000D12F08008A150A1261248A110A164708BF
:102FC000031DDA2F08008A150A1284248A110A16B2
:102FD0004908031DE32F0800B0010330F42FAA3085
:102FE000F22F5530B0000430B8000130B9009820FD
:102FF0008A110A160800000000000000000000000E
:103000008B138B1B002883120317D130E000043090
:10301000E100831203138B17080052288A150A1245
:10302000FD2B8A150A121C2C8A150A12612C8A158E
:103030000A12602C8A150A12842C8A110A1294280A
:103040008A110A127F288A150A12072F8A150A1276
:10305000222F8A150A12F82E8A150A125E2F8A1557
:103060000A1291288A150A1293288A150A1297289B
:103070008A150A12A7288A110A1263288A110A12CD
:10308000052D8A110A1249288A110A125A2A8A1110
:103090000A128A2AA31C5028CD1F50280314512835
:1030A000031008000B088B138B1B5328E8008716AE
:1030B0000511851220086F280B088B138B1B5D28C8
:1030C000E80087160515851221086F280B088B1359
:1030D0008B1B6728E80087160511851622086810E3
:1030E0008316031386018312031386008712871643
:1030F0008316031386098312031305158516871299
:103100000000060868088B008A110A12C12F1830C7
:103110008A0041088207BE28A828A329A329A32939
:10312000A329A329A329A329A329D929C528882903
:10313000F029A828F629272A4A295829A828A828A2
:10314000A828A828A828A828A828A828A828C128E6
:103150008A150A1203306F02031900298A110A1610
:1031600005306F020319A52A8A110A1602306F0270
:103170000319042D0A306F020319042D8A110A1253
:10318000F62D96268A110A12872E01306F02031D32
:103190000829610C031C09290130B000B900033073
:1031A000B80044208A150A16D51B08298330E5008B
:1031B0000130E600A213F71717208A150A160E2011
:1031C0008A150A16031CDC283B208A150A161720CC
:1031D0008A150A1293208A150A1604307D020319F3
:1031E000F428231AE7283E283B208A150A161720C0
:1031F0008A150A1291208A150A1606307D020319D3
:103200000429231AF7283E28D517F713A019A21767
:10321000A828B0010130B9000330B80044208A1555
:103220000A162F208A150A1600307D020319082974
:1032300032208A150A1600307D02031908298330CE
:10324000E500E601A213F71714208A150A160E20CE
:103250008A150A16031C24291720C0248316031379
:10326000B81A4329B81C4329381D43294F1943294B
:10327000831203138A150A1293208A150A16023044
:103280007D02031D2C2983120313D513F713A019F4
:10329000A21708293E0D0639B00061080139B004B3
:1032A0000130B9000030B80044208A150A16A82859
:1032B00096266108033903197829BE008316031383
:1032C0008C12831203132C208A110A1271208A1582
:1032D0000A16051E6E29231A692978298A110A12ED
:1032E0008D208A150A16051A6429231A73297D2947
:1032F0000230BE002C208A150A16831603138C1682
:10330000831203133E0D0639B0006219B00A50292A
:1033100001306F02031DA22914208A150A16853078
:10332000E5004C306102031D9729F0309C29610CA7
:103330004039BF3861057139E6000E208A150A163A
:10334000031C8C29A82801306F020319AF29023011
:103350006F020319AF290A306F02031DD8298A11A1
:103360000A1641208A150A1602306F020319BC2979
:103370000A306F02031DBE294430E1058A150A1286
:1033800061248A150A168030E5006108E600CC3019
:10339000D51BE6050E208A150A16031CBE296108F6
:1033A0000319D529A213F717D829F713A019A217C3
:1033B000A82801306F02031DEF2914208A150A1670
:1033C0008130E50061080339E600FC30D51BE605D5
:1033D0000E208A150A16031CDD296608D029A828A4
:1033E0008A150A16BF268A150A16A82861080F39F9
:1033F000093C031D1F2AA0160D208A150A16E10E8E
:10340000610C04390338E10503191D2A06306102F5
:1034100003181D2A6108430203191D2A61088A1531
:103420000A128B278A150A164308B0000130B9002A
:103430000130B80044208A150A1663102317913012
:10344000E5001130E6000E208A150A16A82823137D
:10345000621A352AA0120D208A150A169130E5004D
:103460001030E6000E208A150A16A828621A362A9D
:103470008B138B1B382A29208A150A1683120317EF
:10348000E830E0000230E100532A621A452A8B132B
:103490008B1B472A29208A150A1683120317D1305D
:1034A000E0000430E100831203138B17621A562ADE
:1034B000621F562AE212231523208A150A16831644
:1034C0000313350883120313BA0083160313360857
:1034D00083120313BB0026208A150A1608007830D1
:1034E000B8000830B90047208A150A16831308303F
:1034F000AF001223B0000130B90077302F07B800B9
:1035000044208A150A1647208A150A16122330020B
:10351000031D6F2AB00944208A150A1647208A1510
:103520000A161223FF3A3002031D6F2AAF0B792AC5
:103530007030B8000530B90047208A150A164330AC
:103540003002031DB32A57303102031DB32A4C3019
:103550003202031DB32A41303302031DB32A4D301A
:1035600034020319D82A4330B0005730B1004C3030
:10357000B2004130B3004D30B4000530B9007030B6
:10358000B80044208A150A16043083120317E31C7E
:10359000CA2A053083120313B0000430B100B2010F
:1035A000B3010430B9000030B80044208A150A166F
:1035B0000030B8000530B90047208A150A1662119C
:1035C00030080139031D6215300C03390319B32A81
:1035D000BE00063031020318B32A31080319B32A9A
:1035E0008A150A128B278A150A160230320203182E
:1035F000B32A9630E5003208031D7717E6000E2047
:103600008A150A16D5133308031DD517631E0F2B11
:10361000771A0F2BAA303402031D0F2B63128A1165
:103620000A12882D1B308A002F038207F134F234EE
:10363000F334F4345F346F347F348F341B308A00BA
:103640002F0882070D340334123403341834033442
:103650001E34033423340334353403343A3403340E
:103660002934033483160313B81A3E280314B81CF4
:103670000310381D03104F190310831203130800A1
:10368000771E432B6316E22517208A110A122E217A
:103690008A150A1686194F2B64080319A8284A2090
:1036A0000318A42CC024322303188E2B9530E50078
:1036B000E6010E208A150A16031C562B4A20031C0D
:1036C000692B621E662B29208A150A160020A31773
:1036D000A828C02483160313B81A3E28B818762BDE
:1036E00083120313D8268A150A165E2B38197E2BEF
:1036F00083120313E1268A150A165E2B4F1D892BB0
:1037000083120313E9268A150A164A20031C822B0A
:103710003E28831203138A110A12B52D8A150A1244
:103720008F208A150A1604307D02031D442B8A154A
:103730000A126A208A150A1606307D02031D442BE0
:10374000E225D51BF62B631AAA2B8A150A12CF2362
:103750008A150A1614208A150A164A200318A42C62
:10376000C0243223031C562B2F208A150A16023040
:103770007D02031DAA2B621AAA2B631ACA2B621E92
:10378000C42B29208A150A1600208A150A12D12373
:103790008A150A1614208A150A164A200318A42C22
:1037A000C0243223031C562B32208A150A160230FD
:1037B0007D02031DCA2B621ACA2BC0243223031CAC
:1037C000562B35208A150A1690307D05031DDD2BFA
:1037D000C0243223031C562B35208A150A164A2092
:1037E0000318A42CA0307D05031DE82BE225E31B64
:1037F000342C631A342C8530E5002230E6000E208C
:103800008A110A1278208A150A1614208A150A16B7
:103810004A20031C162C8530E500F030E6000E200F
:103820008A150A1261248A150A16A42C231A052C5B
:103830008530E5006230E6000E208A110A127820F9
:103840008A150A1614208A150A164A2003180B2C0A
:10385000231A222C8530E500F030E6000E208A1570
:103860000A12D3238A150A1617208A150A168330DE
:10387000E5000130E60011208A150A16031C342CDD
:1038800017208A150A164908031D402C8A110A12AE
:10389000C8278A150A1629208A150A16D51B962CC0
:1038A000631AA32C8A150A12D5238A150A168030AA
:1038B000E5000130E600B0240318A42C8A110A1296
:1038C00026208A150A168430E5000130E600B0246F
:1038D0000318A42C621E6F2C29208A150A160020BA
:1038E0008A150A12D7238A150A168030E50002309D
:1038F000E600B0240318A42C8430E5000230E60072
:10390000B0240318A42C621E882C29208A150A16BC
:1039100000208A150A12D9238A110A1278208A15E2
:103920000A1260248A150A16231A8F2C631AA32CF4
:10393000621E9D2C29208A150A1600208A150A125B
:10394000DB238A150A16B827D510FF158A110A122B
:10395000F52D0E208A110A1286208A150A16B42C1B
:103960000E208A150A1620208A150A1260248A154C
:103970000A164A200318BF2C231AB42C031008007F
:10398000A21E6D2D17208A150A1647084907031D28
:10399000C02C83160313381C6D2D8312031335209E
:1039A0008A150A1683160313FD1FD82C4F15612D97
:1039B0007D088839083C0319E62C0314C30D430A1B
:1039C000031DE72CB816B8103811102DC301B8121A
:1039D00003107D1B0314BC0D3C080319B8103C0AEE
:1039E0000319B81403107D180314BD0D3D08031905
:1039F00038113D0A031938150310FD180314BE0DC4
:103A00003E080319B8113E0A0319B81503107D19B1
:103A10000314BF0D3F08031938123F0A0319381663
:103A200038108312031309306F0203196B2D8316AC
:103A30000313B81C612D381D612DB81D4E2DB81112
:103A4000BE018312031314208230E5002530E60006
:103A50008A150A12FD238A150A16031C232D621EDD
:103A6000342D29208A150A160020621A352D621F6E
:103A7000352D232003308A150A12F1238A150A16E0
:103A8000AF000310AF0D4D26BA00AF0A4D26E2126B
:103A90002315BB0026208A150A166F2D381E6D2DA2
:103AA0003812BF018312031314208230E500353031
:103AB000E6008A150A12FD238A150A16031C542DE6
:103AC0002F2D831203136F0883160313BB00831279
:103AD00003130930EF000314702D83120313031036
:103AE000080083160313B81A3E2883120313933079
:103AF000E5000930E60017208A150A160E208A15FF
:103B00000A16031C7B2D17208A150A1611208A1508
:103B10000A16031C832D831603134F1D982D831241
:103B20000313E9268A150A164A20031C912D3E2804
:103B3000831203134A20031CA52D621EA22D2920E7
:103B40008A150A160020A317D52DC0248316031347
:103B5000B818B02D83120313D8268A150A169A2D89
:103B60003819B82D83120313E1268A150A169A2DE7
:103B700083120313E7268A150A16621ABD2D621FE7
:103B8000BD2D8A110A1271208A150A1617208A156E
:103B90000A16231AC62D8A110A162D2C17208A15EB
:103BA0000A1647084907031DCE2D831603133B0849
:103BB000FD000930BB00831203137D08EF008A115A
:103BC0000A12622F621C2B2EE31F1B2ED51C1B2EEC
:103BD000621A1B2E17208A150A169130E500113043
:103BE000E6000E208A150A16031CEA2D17208A15F6
:103BF0000A1647084907031DF62DA0162030BB0002
:103C00000030BA008A150A1233278A110A122D20B1
:103C100007308A150A12F1238A150A16AF0003101D
:103C2000AF0D1E23BA00AF0A1E23BB00E2122620EE
:103C30008A150A16D51062109030E5006408E60077
:103C40000E208A150A16E31B2B2E6408031D2B2E4B
:103C5000631703102C2E031408001E308A00AF03D4
:103C600003102F0D2F0782078A110A12C22F8A15FF
:103C70000A16C1288A150A1232298A110A16D52D68
:103C80008A110A160D2B8A150A12DB2C8A110A16C4
:103C90002C2C8A150A16362A712D1E308A002F0800
:103CA00082071D340034223400342A3400340C1CC2
:103CB000932E0C1083160313B00AB00A3C30300266
:103CC000031C6F2EB001B10A3C303102031C6F2E71
:103CD000B101B20A18303202031C6F2EB2018312F6
:103CE0000313D51D7A2E83160313C0038312031307
:103CF0000319D511DF1E832E83160313CD03831200
:103D000003130319DF12FF1F932E83160313CE0331
:103D100083120313031D932EFF138A150A12EB2639
:103D20008A150A1655158A110A12CC2C831603130C
:103D3000C201C101981CA02EC10F9A2EC20F9A2E4B
:103D4000981CA02E831203130800981BA82E981706
:103D5000831603138C1ABC2E831203131A088316BE
:103D600003138C1683120313181200001816C201D5
:103D7000C00140142730BF00831203130800043031
:103D80006F02031DC52EDF1BD72E610C031CCF2E27
:103D9000A010A015F71FA21762192017D72EA01187
:103DA000A21320130A306F02031DD72EA01408009F
:103DB000621AE02E621FE02E0B308A150A124F2B7A
:103DC0000800621AE02E621FE02E0C30DD2E0D304E
:103DD000DD2E2230DD2E9930E500E6010E208A1519
:103DE0000A1614208A150A129D208A150A16031C29
:103DF000F12E7D080319F12E8A150A129F208A15CB
:103E00000A16031CFC2E7D08B0008A150A12A12098
:103E10008A150A16031C052F7D08B1008A150A129F
:103E2000A3208A150A16031C0E2F7D08B2008A15DE
:103E30000A12A5208A150A16031C172F7D08B30045
:103E40000430B9000530B80044208A110A12872EC8
:103E500041208A150A16A216362F41208A150A1605
:103E6000A216352F41208A150A1622178A110A1226
:103E7000BE278A150A1641208A150A1608005530F1
:103E8000B0000130B9000430B80044208A150A1689
:103E90009430E5000230E6008A110A16C827D127BF
:103EA000A21222138A110A12BE278A150A16172097
:103EB0008A150A1647084907031D572F8230A000AC
:103EC0008A110A12B8278A150A168B138B1B652FC5
:103ED0006400861B682FFD01FC016400861B772FA0
:103EE000861D6B2FFD0F6D2FFC0F6D2F762FFD01A3
:103EF000FC016400861F6D2FFD0F792FFC0F792FB9
:103F0000762F203084008001840A80300402031D53
:103F1000832FA03084008001840F8B2F83171030F3
:103F200084008001840A70300402031D912F9030B8
:103F300084008001840F992F8A110A12052D2030E8
:103F400047020319B62F46084707840030300402A1
:103F5000031CAC2FE0308407831774088000840AA8
:103F600075088000C70AC70A0314B72F031008009A
:103F7000D51BEE2F20208A150A1617208A150A163F
:103F800038208A150A167D083039031DBA2F231AE6
:103F9000C02F8230E5006130E600B0240318EE2F18
:103FA00020208A150A1638208A150A167D0830390D
:103FB000031DD02F32208A150A1604307D02031DFE
:103FC000D02F231AD32F8030E5003030E600A9240B
:103FD0000318EE2F8030E500E601B0240800000051
:103FE00000000000000000000000000000000000D1
:103FF00000000000000000000000000000000000C1
:08400000803F883F813F843FAF
:02400E00F63F7B
:00000001FF
